:100000000C943C020C9459020C9459020C94590221
:100010000C9459020C9459020C9459020C945902F4
:100020000C9459020C9459020C94E8200C94BA21B7
:100030000C94DA1B0C9459020C9459020C9459023A
:100040000C9459020C9459020C9459020C945902C4
:100050000C949D170C94621C0C9459020C94590238
:100060000C9459020C9459020C9459020C945902A4
:100070000C9459020C9459020C9459020C94590294
:100080000C9459020C9459020C9459020C94590284
:100090000C9459020C9459020C9459020C94590274
:1000A0000C9459020C9459020C945902150515052B
:1000B00041054105A905C705DF06DF06D2056B0628
:1000C0007C067C06AC16AE16B316B616B916BC1670
:1000D000BF1627224E2246234E2246239A22BD22B5
:1000E00046231423232329001E001F002000210083
:1000F0002200230024002500260027002D002E00CA
:100100002A0049004B002B0014001A0008001500BB
:1001100017001C0018000C00120013002F00300004
:1001200031004C004E003542040016000700090063
:100130000A000B000D000E000F00330034002800F1
:10014000E1001D001B000600190005001100100051
:10015000360037003800E5005200E000E300E2001E
:100160002C000151E600E400500051004F00000057
:1001700000000000000035003A003B003C003D005C
:100180003E003F0040004100420043004400450063
:100190002A00A9004A0001000100010052000100EC
:1001A0000100010001000100010001000100C15C2B
:1001B0000100AA004D0001000100500051004F0055
:1001C0000100010001000100010001000100010027
:1001D0000100010001000100010001000100A80070
:1001E0000100010001000100A80001000100010060
:1001F0000100010001000100AC00AE00AB000000F6
:1002000000000000000035003A003B003C003D00CB
:100210003E003F00400041004200430044004500D2
:100220002A00A9004A00010001000100520001005B
:10023000010001002400250026000100010001004A
:100240000100AA004D0001000100500051004F00C4
:100250000100010021002200230001000100010033
:1002600001000100010001000100010027001E0043
:100270001F00200001000100A80001000100010092
:100280000100010001000100AC00AE00AB00000065
:10029000000000000000000000000000000000005E
:1002A0000001010203040506080A0C0F1114181CB2
:1002B0002024292E33393F464C535B626A71798181
:1002C0008A929AA2AAB2B9C1C8CFD5DCE1E7EBF015
:1002D000F4F7FAFCFDFEFFFEFDFCFAF7F4F0EBE7A5
:1002E000E1DCD5CFC8C1B9B2AAA29A928A8179714C
:1002F0006A625B534C463F39332E2924201C181464
:10030000110F0C0A08060504030201010000000099
:100310000000000000000A034D00460036003800CF
:1003200000000C03640069003000690062000000F6
:100330000403090409023B00020100A0FA090400B9
:100340000001030101000921110100012240000701
:1003500005810308000109040100010300000009F0
:10036000211101000122B6000705820320000112BD
:10037000010002000000082540684D010101020053
:100380000105010902A10185020901A10005091960
:10039000012908150025019508750181020501094B
:1003A0003009311581257F950275088106093815B8
:1003B00081257F950175088106050C0A3802158193
:1003C000257F950175088106C0C005010980A1013E
:1003D000850319012AB700150126B700950175108C
:1003E0008100C0050C0901A101850419012AA002A0
:1003F000150126A002950175108100C005010906AE
:10040000A1018506050719E029E7150025019508D2
:10041000750181020507190029EF1500250195F0E6
:1004200075018102050819012905950575019102DB
:10043000950175039101C005010906A10105071980
:10044000E029E715002501950875018102950175E0
:100450000881010507190029FF150026FF009506F0
:100460007508810005081901290595057501910296
:10047000950175039101C00011241FBECFEFDAE092
:10048000DEBFCDBF11E0A0E0B1E0EAE8F8E402C0D1
:1004900005900D92AE38B107D9F722E0AEE8B1E091
:1004A00001C01D92A43DB207E1F70E94ED120C9429
:1004B00043240C94000081E0089581E008950C9499
:1004C0005D0208950C9461021F93CF93DF9300D0D7
:1004D00000D01F92CDB7DEB749835A836B8330912A
:1004E000910189819A81311114C0662359F0222328
:1004F00049F00E941C09182F682F89819A810E9457
:10050000C50803C00E94F008182F69817A81812FE5
:1005100004C00E941C0969817A810F900F900F908E
:100520000F900F90DF91CF911F910C945810FC0108
:10053000262F408151816281738184810C946402F1
:1005400081E00895CF93DF93EC0160E00E94970271
:10055000BE01DF91CF910C9462020C949E110C9419
:100560009A1108950E946F070E94B1022FEF84E351
:100570009CE0215080409040E1F700C000000C94C6
:10058000881C0F931F93CF93DF938C0161E00E942F
:100590009702EC01B8010E945F02882309F444C06D
:1005A000B801CE010E949D168823F1F1B801CE0159
:1005B0000E94251A8823C1F1B801CE010E94391882
:1005C000882391F1B801CE010E948119882361F13D
:1005D000F8018281882309F1CB358DE5D807C1F078
:1005E00050F4C115FCE5DF0781F0CF3DDC45A9F4EF
:1005F0000E94530E19C0CC35EDE5DE0761F0CD3514
:10060000DD4559F40E94960D08C00E94B2020CC04C
:100610000E949F0D02C00E94A20DC801DF91CF91E0
:100620001F910F910C945B0280E0DF91CF911F919D
:100630000F9108950E94BC1B80E00E9455170C94F6
:1006400038030E94C1150E943B030C94C21B0895FD
:100650000C94270381E008950C942A030895CF9306
:10066000C82F0E9428038C2F0E942C03CF9108953D
:1006700080E00C942F030E94811A0C942F030E9497
:10068000811A90919001891721F0809390010C9428
:100690002F030895CF93DF93CDB7DEB72B970FB617
:1006A000F894DEBF0FBECDBF4F83588769877A8726
:1006B0008B8761110E94E20C9E012F5F3F4F86E005
:1006C000F90111928A95E9F785E0FE013796D90183
:1006D00001900D928A95E1F789819A814C815D8123
:1006E000452B31F09F3F31F491E08F3F19F403C067
:1006F00091E001C090E090FF09C049815A816B816F
:100700007C818D819E810E94030C05C0C9010E94DD
:10071000A0028111F2CF2B960FB6F894DEBF0FBE68
:10072000CDBFDF91CF910895FC01808191810E941E
:100730005E090895CF93882309F4A4C0C82F823896
:10074000C1F40E94811A81FD9DC069E3809102017C
:10075000909103010E94771B0E94040D2FEF81EE00
:1007600094E0215080409040E1F700C0000069E330
:1007700019C0833801F50E94811A80FD83C063E5AA
:1007800080910201909103010E94771B0E94040D49
:100790002FEF81EE94E0215080409040E1F700C0BF
:1007A000000063E580910201909103010E94821B89
:1007B000CF910C94040D8438C1F40E94811A82FDFB
:1007C00061C067E480910201909103010E94771B50
:1007D0000E94040D2FEF81EE94E021508040904064
:1007E000E1F700C0000067E4DDCF8CEF8C0F813AA9
:1007F000D0F46C2F80910201909103010E94F71AAE
:10080000882349F06C2F80910201909103010E948E
:10081000821B0E94040D6C2F8091020190910301B4
:100820000E94771BC5CF80E28C0F883048F4C770D8
:1008300081E001C0880FCA95EAF70E94C50CB8CFC5
:10084000EBE5EC0FE33040F4F0E0E75BFE4F808136
:1008500090E0CF910C94B51AE8E5EC0FE73150F435
:10086000F0E0EE0FFF1FE55EFE4F80819181CF919A
:100870000C94CB1ACD3E30F08C2F0E947213CF9186
:100880000C944414CF910895882309F464C08238ED
:1008900079F40E94811A81FF5EC069E380910201B0
:1008A000909103010E94771B0E94040D69E310C020
:1008B0008338B1F40E94811A80FF4DC063E58091B6
:1008C0000201909103010E94771B0E94040D63E5D1
:1008D00080910201909103010E94821B0C94040DEF
:1008E000843879F40E94811A82FF35C067E48091D0
:1008F0000201909103010E94771B0E94040D67E49E
:10090000E7CF9CEF980F913A10F4682FE1CF90E277
:10091000980F983050F4877091E001C0990F8A9534
:10092000EAF7892F0E94CB0CD9CF9BE5980F933023
:1009300020F480E090E00C94B51A98E5980F973178
:1009400020F480E090E00C94CB1A8D3E20F00E94C1
:10095000CD130C94441408951F93CF93DF93182F55
:10096000EB010E949A03209741F08FE99FE00197E5
:10097000F1F700C000002197F6CF812FDF91CF91D2
:100980001F910C944404893319F060E070E002C0B8
:1009900060E570E00C94AC04882321F00E94C50C43
:1009A0000C94040D0895882321F00E94CB0C0C9424
:1009B000040D0895CF92DF92EF92FF920F931F9351
:1009C000CF93DF937C01D62FC72FFC0112810581C5
:1009D00002950F700E94BB0C8823B9F01123A9F077
:1009E0008C2F807F803421F080E28D0F883068F07A
:1009F0008091A10282FD09C082E00E94640D0E94E4
:100A0000BB0C91E0D82ED92601C0D12CCC2EC2949B
:100A10008FE0C8228C2D90E08C30910508F0CFC17A
:100A2000FC01EA5AFF4F0C94D4238C2F807FCF70A7
:100A3000882311F0C295C07F112399F0CC2309F4CB
:100A4000AAC180E28D0F883010F0D11104C08C2F24
:100A50000E94C50C03C08C2F0E94D50C0E94040D6F
:100A60009AC18D2F0E944404CC2309F4A8C180E2CE
:100A70008D0F883038F1DD2329F18C2F0E94DB0C9B
:100A800024C08C2F807FCF70803211F0C295C07F40
:100A9000DD2319F0D130A1F13DC08091A10282FF88
:100AA00017C0112349F0CC2329F08C2F0E94C50CCC
:100AB0000E94040D80E070C180E00E944404CC23B9
:100AC00009F47DC18C2F0E94CB0C0E94040D77C1CC
:100AD000112371F0002341F0013031F40E94E50C44
:100AE0008C2B0E94ED0C6BC10E94E50C8C2B1DC061
:100AF000002319F0013009F462C10E94FA0C25C0EC
:100B0000112321F0063008F05AC10EC0053008F05C
:100B100056C11BC0112361F0002331F0F70185811C
:100B200080FF39C18F7085838C2F0E94CC0447C110
:100B3000002359F0D93309F03FC1FFEF07EE13E06E
:100B4000F15000401040E1F735C18C2F0E94D304D2
:100B500036C18C2F86958695837019F0813061F0AF
:100B60002EC1112321F08D2F9C2F937002C080E0A5
:100B700090E00E94B51A2BC1112321F08D2F9C2FDC
:100B8000937002C080E090E00E94CB1A20C18D2FAC
:100B9000112319F00E94721302C00E94CD130E940B
:100BA000441415C18C2F837009F047C011110BC17B
:100BB0002D2F229526952770220F220F6D2F6F70F3
:100BC000862F90E0A0E0B0E0022E04C0880F991FAD
:100BD000AA1FBB1F0A94D2F7D4FF10C04FE050E009
:100BE00060E070E004C0440F551F661F771F2A9510
:100BF000D2F7409550956095709503C040E050E065
:100C0000BA01C695C695C3708A019B01082B192BA2
:100C10002A2B3B2BC901B801C23049F058F4C1302E
:100C200019F00E94DB07CFC00E94C907CCC00E9408
:100C3000ED07C9C00E94C707C6C0112319F08C2F49
:100C4000817001C08695882309F4BDC02D2F22959F
:100C500026952770220F220F6D2F6F70862F90E040
:100C6000A0E0B0E0022E04C0880F991FAA1FBB1F8E
:100C70000A94D2F7D4FF10C04FE050E060E070E07B
:100C800004C0440F551F661F771F2A95D2F7409561
:100C900050956095709503C040E050E0BA01C6954C
:100CA000C695C3708A019B01082B192B2A2B3B2B5D
:100CB000C901B801C23049F058F4C13019F00E949E
:100CC000A00881C00E948E087EC00E94B2087BC02E
:100CD0000E94010878C0CF70112339F08C2F0E9438
:100CE00027088D2F0E94CC046EC08D2F0E94D30444
:100CF0008C2F0E94480867C0D23F21F128F4D03FD2
:100D000041F0D13FC1F043C0D33F19F1D43F79F056
:100D10003EC0112341F0053008F051C08C2F8F7177
:100D20000E946D084CC0063008F049C0F7CF809192
:100D3000A10282FF18C0112339F08C2F8F710E94FD
:100D400027083DC01123C9F38C2F8F710E944808DA
:100D500036C0112329F08C2F8F710E9412082FC0EA
:100D60000E940D082CC0112349F0CF718C2F0E94D6
:100D7000270863E08C2F0E94490D21C081E00E946A
:100D8000640D0230E0F082E00E94640D18C011236F
:100D900031F0002391F28D2F0E949A0310C000239E
:100DA00099F2D93349F41FEF27EE33E01150204078
:100DB0003040E1F700C000008D2F0E94440488EF0E
:100DC0008C0D843020F40E94811A0E942F03DD20B4
:100DD000C9F00E94B70C80FD15C0F70112820E9475
:100DE000B10C0E942708C7010E9423070E94B10C82
:100DF000DF91CF911F910F91FF90EF90DF90CF90F7
:100E00000C944808DF91CF911F910F91FF90EF90C4
:100E1000DF90CF9008950F931F93CF93DF93EC0152
:100E2000688179818A810E9469098C010E94C408C5
:100E30000E94B507B801CE010E94DA04DF91CF917C
:100E40001F910F910895CF93DF93EC0198818981D1
:100E50002B813C81232B31F08F3F31F481E09F3F88
:100E600019F403C081E001C080E080FD1DC0CE0107
:100E70000E94C102811110C00E94BB0C8823A1F006
:100E80008A81882389F08091A10282FD0DC082E0D1
:100E9000DF91CF910C94640DCE010E940B07CE011F
:100EA000DF91CF910C94A202DF91CF91089580E061
:100EB00090E00E94B51A80E090E00E94CB1A0E9458
:100EC000E20C0E94040D0E9475150C94441480914C
:100ED0000201909103010E948D1B0C9457070E9400
:100EE000D20C0C94670792959F70963079F010F4AD
:100EF000925001C09A50923068F4803F69F018F423
:100F0000883E40F409C0843F29F406C0883E20F0A2
:100F1000813F11F080E0089581E00895FC01808117
:100F200091810E945E090E9473070895CF93DF9319
:100F300000D000D01F92CDB7DEB70F900F900F906A
:100F40000F900F90DF91CF910895CF93DF9300D052
:100F500000D000D0CDB7DEB726960FB6F894DEBF2E
:100F60000FBECDBFDF91CF910895089508950C94E1
:100F7000B6070C94B7070E94B9076093C30170933A
:100F8000C4018093C5019093C6010C9457070C943B
:100F9000BB070F931F930091C3011091C4012091CF
:100FA000C5013091C601602B712B822B932B1F91B1
:100FB0000F910C94BB070F931F930091C3011091E5
:100FC000C4012091C5013091C601602371238223A1
:100FD00093231F910F910C94BB070F931F930091C4
:100FE000C3011091C4012091C5013091C601602751
:100FF0007127822793271F910F910C94BB070C94A4
:10100000B6070E94FF076093BF017093C0018093F1
:10101000C1019093C2010C94570760E070E0CB01CE
:101020000C9401080F931F9341E050E060E070E0E2
:101030008A019B0104C0000F111F221F331F8A95D4
:10104000D2F7C901B8011F910F910C9401080F93B9
:101050001F9341E050E060E070E004C0440F551F72
:10106000661F771F8A95D2F78091BF019091C001CA
:10107000A091C101B091C2018A019B01082B192BDB
:101080002A2B3B2BC901B8011F910F910C94010829
:101090000F931F9341E050E060E070E004C0440F04
:1010A000551F661F771F8A95D2F74095509560951A
:1010B00070958091BF019091C001A091C101B09144
:1010C000C2018A019B01082319232A233B23C9015A
:1010D000B8011F910F910C9401080F931F9341E0E9
:1010E00050E060E070E004C0440F551F661F771F9A
:1010F0008A95D2F78091BF019091C001A091C10162
:10110000B091C2018A019B01082719272A273B2792
:10111000C901B8011F910F910C9401080F931F93FF
:101120000091BF011091C0012091C1013091C20115
:10113000602B712B822B932B1F910F910C94010824
:101140000F931F930091BF011091C0012091C10125
:101150003091C20160237123822393231F910F9149
:101160000C9401080F931F930091BF011091C001CF
:101170002091C1013091C2016027712782279327F6
:101180001F910F910C940108089529E0929F800D02
:101190001124E82FE695E695E695877051E001C0A9
:1011A000550F8A95EAF785E0E89FF0011124EE5685
:1011B000FE4F20E030E070E04081CB01022E02C003
:1011C000969587950A94E2F7817081958427852307
:1011D000842781932F5F3F4F2530310569F70895AC
:1011E00029E0929F800D1124682F6695669566957B
:1011F000982F977085E0689FB001112440E050E07F
:1012000080E0FB01E40FF51FEE56FE4F208130E039
:10121000092E02C0369527950A94E2F721703327EC
:10122000042E01C0220F0A94EAF7822B4F5F5F4F12
:101230004530510531F70895BF92CF92DF92EF927A
:10124000FF920F931F93CF93DF938C01C090BF0148
:10125000D090C001E090C101F090C2018091C30123
:101260009091C401A091C501B091C601C82AD92AA4
:10127000EA2AFB2ACFE1D0E0D701C6010C2E04C038
:10128000B695A795979587950A94D2F780FD04C0E7
:10129000219790F7B12C07C0BC2EB8018C2F0E946B
:1012A0006B100197A9F38B2DDF91CF911F910F91B7
:1012B000FF90EF90DF90CF90BF900895CF93DF9392
:1012C000EC010E941C09BE010E946B10DF91CF91BE
:1012D00008951F93CF93DF93EB0190919101992390
:1012E00021F0CB010E945E0913C0882349F0CB0195
:1012F0000E941C09182F682FCE010E94C50804C047
:10130000CB010E94F008182FBE01812F0E946B10A4
:10131000DF91CF911F9108951F93CF93DF93C091D9
:10132000C70116E08091C801C81799F0D0E01C9F52
:10133000F0011D9FF00D1124E753FE4F40815181B4
:1013400062817381848195810E94A5072196C7706F
:10135000E9CFDF91CF911F9108954091F90150910C
:10136000FA016091FB017091FC018091FD01909167
:10137000FE010C94A507EF92FF920F931F93CF935A
:10138000DF938091FE0182958F7009F065C0809196
:10139000FB01882309F460C08091C701F090C80167
:1013A0001091F9010091FA016091FC017091FD0129
:1013B00091E01F3F09F090E0C0910001D091010140
:1013C000292F96E0E92E8F1509F446C061157105A5
:1013D00021F00F3F21F030E003C031E001C0322F97
:1013E00090E030FD36C0E89EF001E99EF00D11243A
:1013F000DF01A753BE4F11963C911197301329C0BE
:101400003C91311326C012963C911297311121C0A4
:1014100013964D915C911497461B570B4C175D0723
:10142000C0F48091FE018F7080618093FE01E253D1
:10143000FE4F80818F708061808389EF91E00E94F0
:101440002307DF91CF911F910F91FF90EF900C94A4
:101450008C0901968770B7CFDF91CF911F910F91C3
:10146000FF90EF9008959F92AF92BF92CF92DF923C
:10147000EF92FF920F931F93CF93DF93CDB7DEB719
:1014800061970FB6F894DEBF0FBECDBF8C0185E02B
:10149000F801DE011D9601900D928A95E1F7D801C1
:1014A0001296EC909091F901E091FA012091FC01E3
:1014B0003091FD012115310531F0EF3F31F481E02C
:1014C0009F3F19F403C081E001C080E0B82FB170E4
:1014D0009B2E80FD47C1D8014C9111965C911197CC
:1014E0001396AD90BC90149789EFC82E81E0D82E4A
:1014F000F090FB01B501621B730B2091000130914C
:101500000101FF2009F4D9C08091FE016217730721
:1015100008F095C0282F207F09F052C05E1313C039
:10152000491311C0FE2CE1100EC08F7080618093B2
:10153000FE010E94AD09C6010E9423078091FE01B1
:10154000F80185834DC1AB2831F05F3F31F481E074
:101550004F3F19F403C081E001C080E080FD03C06B
:1015600081E08E2502C080E090E0F82FF170FF2E20
:1015700080FF1CC08091C7012091C80136E082170E
:1015800009F40BC190E0389FF001399FF00D112450
:10159000E753FE4F6181561306C06081461303C0B6
:1015A0006281E61203C001968770E9CFFE2CEE201F
:1015B00009F416C18091FE0181608093FE0154C040
:1015C0005E1306C0491304C0E11002C0F80199C0BF
:1015D000C8010E948E07882361F1EE2051F120910D
:1015E000FE01822F82958F7090E0029774F08091B7
:1015F000F9019091FA0198878F831986BB86AA8694
:101600002C87CE0107960E94230786E0F801A9EFF8
:10161000B1E001900D928A95E1F70E94BB090E940A
:10162000AD090AC05E1711F1C8010E948E07811131
:101630002CC0C8010E942307FF24F394D1C0282F97
:10164000207F81F77A2DB98AA88A6E2D89890E9418
:10165000960789EF91E00E94230786E0D6011D924C
:101660008A95E9F70E94AD09F12CBAC04913DCCF85
:10167000E110DACFF8018583C8010E94230786E0D4
:10168000D6011D928A95E9F7ABC0EE2091F2209128
:10169000FE01822F82958F7090E002970CF4B5CFF7
:1016A0008091F9019091FA019A8389831B82BD820E
:1016B000AC822E83CE010196A6CF6217730708F085
:1016C00044C0FE2CEE2009F4B4CF5E1330C04913A1
:1016D0002EC02091FE0120FD21C0822F82958F70A7
:1016E000482F50E041155105C9F0F80125834F30CE
:1016F000510541F08F5F982F9295907F822F8F70C8
:10170000892B8583C8010E94230786E0F801A9EF91
:10171000B1E001900D928A95E1F73CC086E0F801B6
:10172000A9EFB1E001900D928A95E1F759C0C80187
:101730000E948E07811169CF8091FE0181608093A4
:10174000FE01C8010E9423074BC07A2DB98AA88ADE
:101750006E2D89890E94960786E0D6011D928A9592
:10176000E9F718C0EE2009F464CFC8010E948E0783
:10177000F82E882309F45DCF86E0F801A9EFB1E0E7
:1017800001900D928A95E1F789EF91E00E94940310
:101790000E94BB090E94AD0923C04D875E878D85DD
:1017A0009E850E945E09292F22952F70223028F4F1
:1017B0009F7039F0811105C00BC0243028F49F7050
:1017C00049F4805E883020F0C8010E9423079F2CD6
:1017D000F92C06C0D80115969C91907F91F7F8CF0F
:1017E0008F2D61960FB6F894DEBF0FBECDBFDF918F
:1017F000CF911F910F91FF90EF90DF90CF90BF900E
:10180000AF909F9008951F93CF93DF93CDB7DEB72E
:101810002C970FB6F894DEBF0FBECDBF4F8358870D
:1018200069877A878B879C87CE0107960E94330A47
:101830008823D1F09F8188852A853B85232B31F031
:101840008F3F31F481E09F3F19F403C081E001C074
:1018500080E080FD47C04F81588569857A858B85FA
:101860009C850E94A5073EC086E0FE013796DE01FA
:10187000119601900D928A95E1F7FF81E8856A85BE
:101880007B856115710531F0EF3F31F481E0FF3F59
:1018900019F403C081E001C080E080FD23C02091E5
:1018A000C80130E0C9010196877099274091C701AE
:1018B00050E084179507F1F1F983EA837D836C8307
:1018C00096E0929FD001939FB00D1124A753BE4F75
:1018D000FE01319601900D929A95E1F78093C8012F
:1018E0000E948C0916E08091C7019091C801891768
:1018F00071F1189FC001112487539E4F0E94330A33
:10190000882329F1E091C7011E9FF0011124E753BC
:10191000FE4F4081518162817381848195810E9453
:10192000A5078091C70190E0019687709927809361
:10193000C701D9CF0E946F071092C8011092C7014A
:10194000E9EFF1E086E0DF011D928A95E9F72C9638
:101950000FB6F894DEBF0FBECDBFDF91CF911F91C0
:10196000089580911F0285958595859508958091AC
:101970001F028770089590911F02977081E009F40B
:1019800080E0089580914202089590914202892B4F
:10199000809342020895809590914202892380931A
:1019A0004202089510924202089590914102892BBB
:1019B00080934102089580959091410289238093FC
:1019C00041020895109241020895809120020895E5
:1019D00008950C94E80C0C94E90C9091A10292FDEE
:1019E00008C090912002981721F0809320020C9457
:1019F000EB0C089580912002882329F01092200298
:101A000080E00C94EB0C0895CF93DF93E0910201FA
:101A1000F0910301809142028083E0910201F091F4
:101A20000301908180914102892B80838091200263
:101A3000882381F0E0910201F09103019081892BCC
:101A4000808380910201909103010E94E11A81112B
:101A50000E94FA0CC0910201D091030140E250E0D3
:101A60006FEF71E0CE010E94F423892B69F080E2D0
:101A7000FE01AFEFB1E001900D928A95E1F7CE0142
:101A8000DF91CF910C948D1ADF91CF9108950C9432
:101A9000E80C9091A10292FD10C098E0899F9001FE
:101AA0001124262B20931F020E94270880911F02D9
:101AB0008595859585950C94470D0C942708109273
:101AC0001F0280E00C94470D20911F028095822315
:101AD00080931F02982F977099F430E0482F082EBA
:101AE000000C550B2417350759F09091A10292FD77
:101AF00007C08595859585950E9448080C945F0DD3
:101B000008959091A10292FB222720F9281769F0ED
:101B100080FB92F99093A1028091A0029091A10282
:101B20000E94CF0D82E00C94640D08958091A10273
:101B300082FB882780F991E089270C94810D81E050
:101B40000C94810D80E00C94810D6FEF7FEF80E0AD
:101B500090E00C942D2480E090E00E94092421E084
:101B6000893E9E4F09F020E0822F089582E090E0A8
:101B70000C94012483E090E00C940124CF9384E042
:101B800090E00E940124C82F82E290E00E9401248C
:101B90002C2F30E0A901582BCA01CF910895CF9383
:101BA000C92F682F84E090E00E940F246C2F82E2FE
:101BB00090E0CF910C940F24AB01BC018FE090E03A
:101BC0000C942124AB01BC0183E190E00C9421240E
:101BD00060E070E0CB010C94E20D60E070E0CB01BE
:101BE0000E94DC0D0C94E80D69EE7EEF80E090E041
:101BF0000E942D2460E082E090E00E940F2460E0CB
:101C000083E090E00E940F241092C3011092C4015F
:101C10001092C5011092C60160E084E090E00E943D
:101C20000F2460E082E290E00E940F2460E085E0F3
:101C300090E00E940F2460E086E090E00E940F2474
:101C40006FEF87E090E00E940F2440E050E0BA017F
:101C500088E090E00E94212460E08DE090E00E9406
:101C60000F2440E050E0BA0188E190E00E94212476
:101C700060E087E190E00E940F2440E050E0BA016C
:101C80008CE190E00E94212460E070E080E290E02E
:101C90000E942D2440E050E0BA0188E190E00E94CB
:101CA00021240C94ED0D0C94F40D682F8EE090E03F
:101CB0000C940F240E94471C6093570270935802A3
:101CC0008093590290935A02609353027093540286
:101CD0008093550290935602089585B7806885BF1A
:101CE00085B7806885BF089581E008950C94740ECF
:101CF00008950C94780E0C94780E0C947B0E0C9432
:101D0000780E0C947F0E0C94780E0E946D0E87E472
:101D100091E10E94771A0E94830E0C94810E0E941A
:101D2000790E0C94780E0E9461110E942E030C947F
:101D300023180E94321C0E9446120E94930E0E9499
:101D4000C1150C947D0E5F926F927F928F929F923D
:101D5000AF92BF92CF92DF92EF92FF920F931F93B9
:101D6000CF93DF93CDB7DEB72A970FB6F894DEBFD7
:101D70000FBECDBF0E945B12C82E81110E945A0E69
:101D800033E4832E32E0932E00E010E0502E802FBB
:101D90000E9485115C01F401619071904F016826E9
:101DA000792661147104B1F40F5F1F4F08301105DB
:101DB00069F78FEF89838A831B820E943B1C8160B5
:101DC000782F9D838C8349815A816B818D810E94FC
:101DD0004A033AC080915B0281FD0E948E11D12C92
:101DE000EE24E394F12CC3018E219F21892B29F14C
:101DF0000E94760E8823A9F0DE825F82AE20BF208B
:101E000081E0AB2809F480E088870E943B1C816058
:101E1000782F9A8789874E815F8168858A850E949D
:101E20004A03000F111FF801ED5BFD4F8081918186
:101E3000E826F926F182E08207C0D394EE0CFF1C5D
:101E4000F9E0DF12D0CFB0CF81E0C11001C080E057
:101E50002A960FB6F894DEBF0FBECDBFDF91CF91AB
:101E60001F910F91FF90EF90DF90CF90BF90AF90B8
:101E70009F908F907F906F905F9008950E94A30E27
:101E80000E9487170E9462140C943F03CF93DF9344
:101E90000E947010EC01811521E5920708F045C001
:101EA000811530E5930708F094C0883E910528F528
:101EB000803E910508F0F8C0883A910570F4853AA3
:101EC000910508F07CC08130910509F475C008F4D3
:101ED000E8C0049708F0E8C0E4C08F3B910508F023
:101EE000E0C0C85AD0E0CC0FDD1FC45BDE4F0990C4
:101EF000D881C02DCE019464D8C0811540E29407EA
:101F000058F4811551E0950708F0CEC08D3E91053B
:101F100008F4C7C09065C9C0C11580E4D80708F4AB
:101F2000C0C0DF70CE01906AC0C0811525E5920760
:101F3000A8F4811534E5930708F095C0811543E5B1
:101F4000940708F07BC0811552E5950708F061C041
:101F5000D82FCC27CE01816F906AA7C0C11589E523
:101F6000D807A0F4C11528E5D20708F082C0C11532
:101F700036E5D30708F095C08C2F0E9404118F71AD
:101F800090E0D82FCC27CE0190628FC0C1154AE5D2
:101F9000D40708F474C0CE0190568115904208F021
:101FA00080C08D2F8F710E940411DD27D0628F7148
:101FB000AE01582BCA0179C081E090E076C0C55AC5
:101FC000D0E0C658DE4F8881C82FD0E0CE019064A3
:101FD0006CC074E0969587957A95E1F7282F237069
:101FE0003C2F337081E090E002C0880F991F3A9532
:101FF000E2F79C68AC01522B9A019C2F9F7096953A
:10200000969550E2959FE0011124C9018C2B9D2BE0
:102010004CC08370992721E030E002C0220F331FAB
:102020008A95E2F79C2F9695969580E2989FE0011D
:102030001124C22BD32BCE019C6837C08370992703
:1020400021E030E002C0220F331F8A95E2F79C2F77
:102050009695969540E2949FE0011124C22BD32BD4
:10206000CE019A6822C0D82FCC27CE01846F906A07
:102070001CC0DC2FCC27CE01806F906A16C08C2F3D
:102080008F700E94041194E0D695C7959A95E1F758
:10209000CF70D0E0DC2FCC27D0699E01282BC9015E
:1020A00004C080E090E001C0CE01DF91CF9108959F
:1020B00028E4829FC0011124FC0129E0729FE00DF9
:1020C000F11D1124E60FF11DEE0FFF1FEA51FF4F26
:1020D0008591949108950E9458100E94460F08958A
:1020E0008238910569F1B0F48133910509F46DC02E
:1020F00048F48932910509F463C08A32910509F4E4
:1021000069C008958533910509F455C08933910557
:10211000B9F00895833E910569F138F4803E910548
:10212000B1F0823E910509F10895863E9105A9F12D
:10213000873E9105B9F1843E910509F064C023C042
:102140002091A00220FD4FC021FD4DC00895809137
:10215000A00280FD44C08091A10280FF44C0809114
:10216000A00284FD42C083EE4DC08091A00282FF98
:1021700038C0F5CF8091A00282FD33C08091A102CA
:1021800080FD31C0ECCF8091A10281FF32C08091EF
:10219000A00284FD2AC087EE35C08091A00283FF93
:1021A00026C0F5CF8091A00283FD21C08091A102BD
:1021B00081FD1FC0ECCF8091A00285FD1CC01DC019
:1021C0008091A00285FD19C016C08091A00286FDF5
:1021D00016C017C08091A00286FD13C010C089E30D
:1021E00011C082EE0FC080EE0DC080E00BC086EE05
:1021F00009C084EE07C089E205C085E303C08AE216
:1022000001C081E390E008959091A00292FF0DC07B
:10221000282F2871283019F4877F846006C0282F62
:102220002471243011F48B7F886093FF0DC0282F18
:102230002871283119F4877E846106C0282F247103
:10224000243111F48B7E88612091A10220FF0DC002
:10225000382F3871383019F4877F816006C0382FE5
:102260003171313011F48E7F886021FF0DC0282F2D
:102270002871283119F4877E816106C0282F2171C9
:10228000213111F48E7E886194FD877E089580E06F
:1022900008950C94A50D0E945B128FE39CE90197B1
:1022A000F1F700C000000E945B1280E00E948511DF
:1022B00080FF04C00E9449110C94881C08950C945E
:1022C0004B110E94AB0D811102C00E94530E0E945F
:1022D000B60D80935B020E94BE0D9093A102809385
:1022E000A0020E945F110E94BA0D682F70E080E08A
:1022F00090E00E94C7076091BF017091C00180917A
:10230000C1019091C2010C94FF07E82FF0E0EE0F9D
:10231000FF1FEE54FD4F808191810895089580EA5A
:102320008A95F1F7089500C008950C948F110895CF
:102330000C9497110C9498110C9497110C949C1177
:10234000F894E82FE295EF70F0E031A1282F2F707C
:1023500081E090E001C0880F2A95EAF7982F9095C8
:10236000932391A392A1892B82A3789408950F932C
:102370001F93CF93DF93C6E8D1E089918F3F11F08F
:102380000E94A01181E0CE38D807B9F7CDE7D1E09F
:1023900006E811E089918F3F11F00E94A0110C17FF
:1023A0001D07C1F7DF91CF911F910F910895BF9243
:1023B000CF92DF92EF92FF920F931F93CF93DF9311
:1023C0008C01C62FD0E0CE018A579E4F6C01FC01D4
:1023D00090819F3F09F450C0B62EF894E92FE29502
:1023E000EF70F0E081A19F7021E030E001C0220F8A
:1023F0009A95EAF7822B81A382A12095282322A314
:1024000078940E949311EDE7F1E046E851E021E075
:1024100030E0E12CF12C61916F3F89F0A62FA2955D
:10242000AF70B0E090968C9190E06F7002C095957F
:1024300087956A95E2F780FD02C0C90102C080E07D
:1024400090E0E82AF92A220F331F4E175F0719F789
:10245000F60180818F3F11F00E94A01161E0E1142C
:10246000F10409F460E08B2D0E949511CC0FDD1F63
:10247000C00FD11FF982E882DF91CF911F910F9198
:10248000FF90EF90DF90CF90BF9008950E94B7111A
:1024900080E1E2EBF2E0DF01982F1D929A95E9F7D7
:1024A000E2EAF2E0DF011D928A95E9F788E00E94F6
:1024B000A6120C94AD02FF920F931F93CF93DF935C
:1024C000CDB7DEB760970FB6F894DEBF0FBECDBFB5
:1024D0008E010F5F1F4F80E1F80111928A95E9F795
:1024E000F12C6F2DC8010E94D711F394F8E0FF1270
:1024F000F8CF40E150E0B80182EA92E00E94F42374
:10250000FF24F394009709F4F12C892B41F080E12A
:10251000F801A2EAB2E001900D928A95E1F72F2D21
:1025200048E062EB72E082EA92E00E94A7120E9409
:10253000AF028F2D60960FB6F894DEBF0FBECDBFF1
:10254000DF91CF911F910F91FF9008950895FF9211
:102550000F931F93CF93DF93F82E092F162FD72FAA
:10256000C42F222349F081E080935E020E943B1C2D
:1025700090935D0280935C0280915E028823D9F083
:1025800080915C0290915D020E94531C059798F027
:10259000EF2DF02FA12FBD2F80E090E04C2F50E0C9
:1025A0008417950734F4219131912D933D93019631
:1025B000F7CF10925E02DF91CF911F910F91FF90A4
:1025C00008950E94401E0E94990E0C944C1E0E9479
:1025D000501E0E943E0F0C946A1E0E94D91B0E943E
:1025E000271E0E94850E0E94E1120E94E7120E949F
:1025F0008F0EFBCF8091650280FF06C060910901BC
:1026000070E0660F771F26C081FF04C0609109014A
:1026100084E005C082FF07C06091090188E0689FDF
:10262000B001112417C0909164029923D1F06091F8
:102630000801961788F72091090188E0289F9001EA
:102640001124929FA001939F500D112470E0CA01A4
:102650000E949E236038710540F46115710519F4DC
:1026600006C068E070E0862F08958FE7089581E046
:1026700008958091650280FF08C06091050170E0B7
:10268000759567957595679521C081FF06C0609126
:10269000050170E07595679519C082FF04C06091CF
:1026A000050170E010C090916302992399F0609148
:1026B00004019617A0F780910501899FC00111249C
:1026C00070E00E949E236038710540F46115710529
:1026D00019F406C061E070E0862F08958FE7089531
:1026E00081E008958D3E21F40E94FA12819504C084
:1026F0008E3E29F40E94FA128093690208958F3E5B
:1027000021F40E94FA12819504C0803F29F40E94AE
:10271000FA12809368020895893F19F40E943913D0
:1027200005C08A3F31F40E943913819580936A0273
:1027300008958B3F21F40E943913819504C08C3F8A
:1027400029F40E94391380936B0208959FE0980F3B
:10275000983078F421E030E0A90102C0440F551F01
:102760009A95E2F7CA0190916702892B80936702DC
:1027700008958D3F21F48091650281600BC08E3FEA
:1027800021F480916502826005C08F3F29F4809119
:10279000650284608093650208958D3E39F49091BE
:1027A000690297FF35C01092690259C08E3E29F424
:1027B000909169021916BCF32BC0909168028F3E6C
:1027C00029F497FF25C01092680249C0803F19F490
:1027D0001916CCF31DC090916A02893F29F419168D
:1027E000BCF410926A023BC08A3F19F497FF10C0F4
:1027F000F8CF8B3F39F490916B0297FF09C010928C
:102800006B022DC08C3F21F490916B021916BCF322
:102810009FE0980F983080F421E030E0A90102C0D9
:10282000440F551F9A95E2F7CA018095909167026F
:1028300089238093670213C08D3F21F48091650244
:102840008E7F0BC08E3F21F4809165028D7F05C085
:102850008F3F29F4809165028B7F80936502809180
:102860006802811106C080916902811102C0109234
:10287000640280916A02811106C080916B0281110D
:1028800002C01092630208950E943B1C20916802CE
:10289000211104C020916902222321F09093620249
:1028A0008093610220916A02211104C020916B0281
:1028B000222321F09093600280935F0286E692E0EB
:1028C0000C94A71AEF92FF920F931F93CF93DF936D
:1028D00000D000D000D0CDB7DEB786E0E6E6F2E06B
:1028E000DE01119601900D928A95E1F7E090680261
:1028F000F090690200916A0210916B0210926802D6
:102900001092690210926A0210926B02E11003C0E9
:10291000FF2009F45DC080916102909162020E94E3
:10292000531CAC0190916402992339F020910A0163
:1029300030E02417350758F04BC020910B018AE096
:10294000289F900111242417350718F041C09F3F9C
:1029500019F09F5F90936402EE2061F00E94FA12DA
:102960001E1414F09FEF01C091E0989F902D112448
:1029700090936802FF2061F00E94FA121F1414F075
:102980009FEF01C091E0989F902D112490936902D0
:10299000309168023323E1F0209169022223C1F0D3
:1029A00045EB3403C0011124992319F09093680278
:1029B00003C081E08093680235EB2303C00111243A
:1029C000992319F09093690203C081E08093690212
:1029D000011103C0112309F45DC080915F02909141
:1029E00060020E94531CAC0190916302992339F05C
:1029F0002091060130E02417350758F04BC0209194
:102A000007018AE0289F900111242417350718F048
:102A100041C09F3F19F09F5F90936302002361F0D4
:102A20000E943913101614F09FEF01C091E0989F97
:102A3000902D112490936A02112361F00E943913A2
:102A4000111614F09FEF01C091E0989F902D112472
:102A500090936B0230916A023323E1F020916B0274
:102A60002223C1F045EB3403C0011124992319F04E
:102A700090936A0203C081E080936A0235EB2303DE
:102A8000C0011124992319F090936B0203C081E0D7
:102A900080936B028091680281110BC08091690262
:102AA000811107C080916A02811103C080916B027D
:102AB00081110E944414EB82FC820D831E8386E008
:102AC000FE013196A6E6B2E001900D928A95E1F7FB
:102AD00026960FB6F894DEBF0FBECDBFDF91CF9123
:102AE0001F910F91FF90EF900895E6E6F2E086E0E7
:102AF000DF011D928A95E9F7109264021092630239
:102B000010926502089586E090E00C940124682FED
:102B100086E090E00C940F248091C2028470896159
:102B20008093C2020C9487158091C2028695869587
:102B3000869508958091C20281FD07C082608093CE
:102B4000C2020E9487150C94881708958091C202D2
:102B500081FF07C08D7F8093C2020E9487150C946D
:102B6000941708958091C20281FD0C94A6150C94CF
:102B70009A158091C20286958170089580910C010A
:102B800008950E94AB0D811104C00E94530E0E9453
:102B90008C150E9483158093C202282F26952695B6
:102BA000269530E02430310524F0877088618093C9
:102BB000C2028091C20280FF04C0869586958695E8
:102BC00001C080E00C9455172091C202822F869597
:102BD00086958695482F50E04330510554F48F5F19
:102BE000982F990F990F990F822F8770892B8093B7
:102BF000C2028091C20281608093C2020E94871546
:102C00008091C2028695869586950C945517809181
:102C1000C202982F969596959695A1F0915E990F80
:102C2000990F990F8770892B8093C202887F91E05A
:102C300009F490E08091C20290FB80F98093C20277
:102C40000E9487158091C2028695869586950C9480
:102C500055178091C20280FD13C081608093C2022B
:102C6000813019F489E08093C2028091C2020E94EF
:102C700087158091C2028695869586950C94551786
:102C800008958091C20280FF08C08E7F8093C202A7
:102C90000E94871580E00C94551708958091C20218
:102CA00080FD0C9441160C9429169091C202892F34
:102CB0008695869586958F5F8F719770843038F4EE
:102CC000880F880F880F892B8093C20202C09093CF
:102CD000C2028091C202887F91E009F490E0809165
:102CE000C20290FB80F98093C2020E9487158091F6
:102CF000C2028695869586950C945517843008F007
:102D000083E09091C2029770282F220F220F220F8A
:102D1000922B9093C202987F21E009F420E09091D9
:102D2000C20220FB90F99093C2020C9455170E94A6
:102D30007E168091C2020C948715FC01DB0112966D
:102D40008C918823F9F0EC5BFC45E730F105D8F471
:102D5000EE59FF4F0C94D42383E001C080E00E9421
:102D6000971680E008950E940716FBCF0E94E41595
:102D7000F8CF0E944E16F5CF0E945516F2CF0E9452
:102D8000B215EFCF81E00895259A2D9808952D98DA
:102D900008958F929F92AF92BF92CF92DF92EF925F
:102DA000FF920F931F93CF93DF938C018091860046
:102DB000909187006CE070E00E948A236017710791
:102DC00030F0C80169E070E00E948A2360C0809101
:102DD000860090918700E0908600F0908700E09157
:102DE0008600F0918700C6E0D0E0BE010E948A23F1
:102DF00020E030E0060F171F211D311D4801590149
:102E000085E0880C991CAA1CBB1C8A95D1F7C701C8
:102E1000BE010E948A236F01E12CF12CA7019601CB
:102E2000260F371F411D511DC501B4010E94B22359
:102E300069017A01E0918600F0918700CA01B90129
:102E40000E947A239B01AC01DF010E94E9239B01D0
:102E5000AC01C701B6010E947A23DC01CB012FE04F
:102E6000B695A795979587952A95D1F700918600F5
:102E70001091870020E030E0081719072A073B0768
:102E800028F46091860070918700CB01BC01CB01D2
:102E9000DF91CF911F910F91FF90EF90DF90CF9036
:102EA000BF90AF909F908F900895CF93C82F84309C
:102EB00050F4811109C0809180008F778093800049
:102EC0000E94C71606C0C3E080918000806880938E
:102ED0008000A0918600B09187002C2F30E00E94E6
:102EE000DA2323E030E040E050E00E94B223B42F28
:102EF000A32F922F8827892F9A2FAB2FBB270E94B1
:102F0000C9169093890080938800CF910895089501
:102F100010926D0210926C0210926E02EFE6F0E0D9
:102F20008081816080830895EFE6F0E080818E7F6C
:102F300080830E9494150C9455171F920F920FB620
:102F40000F9211240F931F932F933F934F935F93EF
:102F50006F937F938F939F93AF93BF93CF93EF9391
:102F6000FF9380910D0191E0980F823019F09093BA
:102F70000D0155C081E080930D010E94BE15C82F40
:102F800000916C0210916D020F5F1F4F0E94BE15E1
:102F900028E7829FB0011124C8010E948A239093E0
:102FA0006D0280936C0228E7C29FB0011124660F66
:102FB000672F661F770B71950E948A236F77809128
:102FC0006E02823019F4603451F404C0813039F457
:102FD0006F3729F480916F008E7F80936F00E62F0A
:102FE000F0E0EA56FD4FC4910091860010918700F1
:102FF0000E949415282FC09FC001C19F900D1124DD
:103000006DEF72E00E948A23269FC001279F900DDA
:1030100011240E94C9169093890080938800FF9123
:10302000EF91CF91BF91AF919F918F917F916F91D0
:103030005F914F913F912F911F910F910F900FBE74
:103040000F901F9018950E94C41682E8809380000C
:1030500089E1809381008FEF9FEF909387008093A9
:1030600086000E94C1150E94B91581110C94881721
:103070000895CF93DF93EC01FB018281882309F44B
:103080003CC1C430FDE5DF0760F4CB3F9CE5D907C8
:1030900088F49E0122503C452431310508F02EC1B0
:1030A00009C0C236EDE5DE0729F0C63AFDE5DF07C7
:1030B00009F024C10E94BE0D9093A1028093A0024A
:1030C000C1318CE5D80709F4C6C008F042C0C93048
:1030D000ECE5DE0709F49BC000F5C5308CE5D807A8
:1030E00009F485C078F4C330ECE5DE0709F478C054
:1030F00008F07AC0C230DC4509F0F5C08091A0022A
:103100008160EFC0C7309CE5D90709F478C008F0AA
:103110007AC08091A0028061E4C0CD30FCE5DF0779
:1031200009F487C058F4CB309CE5D90709F479C07D
:1031300008F07BC08091A00288606FC0CF30FCE5B2
:10314000DF0709F480C008F082C08091A002877F69
:10315000C8C0CE3F9CE5D90709F471C000F5C53160
:10316000FCE5DF0709F485C068F4C3319CE5D907A5
:1031700009F475C008F095C00E946F078091A00205
:103180008F77AFC0CC3FFCE5DF07A9F108F054C052
:10319000CB3FDC4509F0A7C08091A10240C0C230FE
:1031A000EDE5DE0709F489C058F4C1158DE5D807AF
:1031B00009F45AC008F069C08091A10282602FC052
:1031C000C236EDE5DE0709F47CC0C63AFDE5DF074F
:1031D00009F481C0C330DD4509F085C080E06EC0D0
:1031E0008091A00282607DC08091A00216C0809173
:1031F000A002886076C08091A10282604FC0809159
:10320000A00280626EC08091A00280646AC00E94A9
:103210006F078091A002806864C0846062C0816092
:103220003DC08091A0028E7F5CC08091A0028D7F06
:1032300058C08091A00216C08091A10218C0809150
:10324000A1028D7F2BC08091A0028F7E4AC0809109
:10325000A0028F7D46C08091A0028F7B42C08091EA
:10326000A002877F8B7F3DC08091A1028D7F8E7FE2
:1032700015C08091A00282FB222720F991E09227BD
:1032800090FB82F990FB83F92CC08091A102982FCA
:10329000909591708E7F892B90FB81F98093A1028C
:1032A00022C00E946F078091A00287FB222720F98D
:1032B00091E0922790FB87F914C081E00E94550E9F
:1032C00012C08091A00284FB222720F991E092276E
:1032D00090FB84F906C08091A002982F909590FBF6
:1032E00080F98093A0028091A0029091A1020E9497
:1032F000CF0D0E946F0780E001C081E0DF91CF9188
:103300000895CF93DF9386319C4541F5EB010E94F0
:10331000C20C982F8A8120910201309103018823E9
:1033200079F09A7A81E009F480E080936F0291113C
:1033300002C069E201C065E3C9010E94771B0AC0AF
:1033400080916F02811102C069E201C065E3C90189
:103350000E94821B0E94040D80E001C081E0DF9189
:10336000CF9108950F931F93CF93DF93C42FD22F44
:10337000FC0182818823C9F0409372020E943B1CA9
:10338000909371028093700280E28C0F883008F075
:1033900057C0C77081E001C0880FCA95EAF7DF9176
:1033A000CF911F910F910C94CC048091720248131D
:1033B00030C080917002909171020E94531C883C31
:1033C000910538F510E21D0FCD17B9F080E28C0F92
:1033D000883040F4C77081E001C0880FCA95EAF7D1
:1033E0000E94D304183028F581E09D2F977001C00A
:1033F000880F9A95EAF70E94CC04802F0E94C3049C
:103400001830F0F4D77081E001C0880FDA95EAF740
:103410000AC080E28C0F883098F4C77081E001C048
:10342000880FCA95EAF7DF91CF911F910F910C9405
:10343000D304802FDF91CF911F910F910C94C3047F
:10344000DF91CF911F910F9108950F939C01CB01B4
:10345000243F4CE5340731F188F4293DFCE53F0772
:10346000D9F02A3D4CE5340779F1283D3C45A9F5D2
:1034700006E221EE41EE68ED7CE52BC0263FFCE53F
:103480003F07E1F0A8F0273F3C4539F507E225EE7C
:1034900046EE67EF7CE51DC007E225EE45EE69EDDF
:1034A0007CE517C006E221EE40EE64EF7CE511C03A
:1034B00007E225EE44EE65EF7CE50BC006E221EE67
:1034C00042EE66EF7CE505C008E221E045EE6AEDDC
:1034D0007CE50E94B21980E008C0FC01828188234B
:1034E00019F01092720201C081E00F91089590933B
:1034F0008F0180938E0108959093780280937702D4
:103500000895E0917702F0917802309721F00190D0
:10351000F081E02D099480E00895E0917702F09128
:103520007802309799F020911A01222359F02091C6
:10353000A00227FF07C0DC012C9111962C93119754
:1035400026E02C930280F381E02D09940895E09108
:103550007702F0917802309739F022E0DC012C9369
:103560000480F581E02D0994089520917502309131
:1035700076022817390771F09093760280937502CE
:10358000E0917702F0917802309721F00680F78180
:10359000E02D099408952091730230917402281748
:1035A000390771F09093740280937302E09177026F
:1035B000F0917802309721F00084F185E02D099494
:1035C0000895FC01329680911A01882331F0809190
:1035D000A00287FF02C09EE101C096E080E091500A
:1035E00028F021912223D9F38F5FF9CF0895662324
:1035F00051F120911A012223E9F02091A00227FF26
:1036000019C0462F4695469546954E31E0F46770B1
:1036100021E030E002C0220F331F6A95E2F7FC017F
:10362000E40FF11D828190E02823392381E0232BD0
:1036300069F409C0FC01329608962191621729F0BD
:10364000E817F907D1F780E0089581E008959C011B
:10365000FC0132969FEF80E04191461789F09F3F31
:1036600019F4411101C0982F8F5F8630A9F79F3F51
:1036700039F0F901E90FF11D97FDFA95628308957C
:1036800008959C012A5F3F4FFC014281461301C00F
:103690001282019682179307B9F70895262F26956F
:1036A000269526952E3168F4FC01E20FF11D677016
:1036B00021E030E001C0220F6A95EAF78281282BD1
:1036C00022830895262F2695269526952E3170F46F
:1036D000FC01E20FF11D677021E030E001C0220F14
:1036E0006A95EAF720958281282322830895209104
:1036F0001A01222329F02091A00227FD0C944E1BD1
:103700000C94271B20911A01222329F02091A0025A
:1037100027FD0C94621B0C94411B20911A01FC01A3
:103720003296222331F08091A00287FF02C08EE101
:1037300001C086E0DF011D928A95E9F7089508959A
:103740000C949F1B83E0809379020C94A01B811141
:1037500002C081E001C082E0809379020C94A01B3A
:103760000C94A71B81E0809379020C94A01B0C940D
:10377000B21B08950C94B91B0C94BA1B0C94B91B82
:103780000C94B91B0C94B91BCF930E94C01B0E94D0
:103790005B120E94BE1BC0E08C2F0E948511892BFA
:1037A00029F4CF5FC830C1F780E001C081E0CF913C
:1037B000089508951F920F920FB60F9211248F93C0
:1037C0009F93AF93BF9380917A02811113C0809130
:1037D000C3029091C402A091C502B091C602419665
:1037E000A11DB11D8093C3029093C402A093C50292
:1037F000B093C602BF91AF919F918F910F900FBE72
:103800000F901F9018958091CB02843031F10E9467
:103810001A0310927A0220E488E190E00FB6F8943F
:10382000A895809360000FBE2093600083B7817FCE
:10383000846083BF83B7816083BF7894889583B7A2
:103840008E7F83BF0FB6F894A89580916000886141
:1038500080936000109260000FBE08950E946F0771
:103860000C94210382E084BD93E095BD9AEF97BD4F
:1038700080936E0008952FB7F8948091C3029091C1
:10388000C402A091C502B091C6022FBF08952FB700
:10389000F8946091C3027091C4028091C502909126
:1038A000C6022FBF08959C014FB7F8948091C302C0
:1038B0009091C402A091C502B091C6024FBF821B75
:1038C000930B089578941F920F920FB60F921124C4
:1038D0008F939F93AF93BF938091C3029091C40243
:1038E000A091C502B091C6020196A11DB11D8093A1
:1038F000C3029093C402A093C502B093C602BF91C5
:10390000AF919F918F910F900FBE0F901F901895C0
:1039100087E797E790930108809300089AE088E191
:103920000FB6F894A895809360000FBE9093600046
:10393000FFCF80919E020895089522E02093E90030
:103940002FEF3091E800215035FD06C035ED3A9556
:10395000F1F700002111F5CF2091E80025FF0BC001
:1039600040E050E066E070E00E94DC1E8091E800DC
:103970008E778093E8000895CF93DF9320911A010A
:10398000222339F02091A00227FF03C060E222E049
:1039900002C068E021E02093E9002FEF3091E800B9
:1039A000215035FD06C035ED3A95F1F700002111A3
:1039B000F5CF2091E80025FF1DC0EC0180911A0190
:1039C000811105C040E050E068E070E003C070E0A5
:1039D00040E050E0CE010E94DC1E8091E8008E772E
:1039E0008093E80080E2FE01AEE7B2E001900D9224
:1039F0008A95E1F7DF91CF91089580937B027093D0
:103A00007D0260937C028091CB02843001F582E0DC
:103A10008093E9008FEF9091E800815095FD06C0FA
:103A200095ED9A95F1F700008111F5CF8091E800AE
:103A300085FF0DC040E050E063E070E08BE792E06E
:103A40000E94DC1E8091E8008E778093E800089544
:103A5000BC0184E00C94FD1CBC0183E00C94FD1CB3
:103A60008091CA02811109C00E946D200E94CA2063
:103A70008091E20084608093E20008951092CA026F
:103A800008950C94B71B6091C70281E0611101C0D9
:103A900080E00C94A21B9091CB0281E0943009F05D
:103AA00080E06091C7020C94A71B42E061EC81E0CA
:103AB0000E94E61F42E261EC82E00E94E61F9091C4
:103AC000CB0281E0943009F080E06091C7020C9451
:103AD000B01B8091CD02833009F461C030F4813095
:103AE00071F0823009F49AC008958A3009F486C0D2
:103AF0008B3009F46CC0893009F0A8C020C08091D7
:103B0000CC02813A09F0A2C08091E800877F8093BF
:103B1000E8008091D0029091D102892B21F460E2DB
:103B20008EE792E003C060E080E090E070E00E94E9
:103B3000271F8091E8008B778093E800089580919B
:103B4000CC02813209F082C08091D0029091D102E2
:103B5000029708F07BC08091E800877F8093E8009F
:103B60008091E80082FD05C08091CB028111F8CFE1
:103B70006DC02091F3008091F20090E0922B0297AB
:103B800031F48091F100813011F0863021F4809180
:103B9000F10080939E028091E8008B7753C0809162
:103BA000CC02813A09F052C08091D0029091D102AA
:103BB000892B09F04BC08091E800877F8093E80053
:103BC0008091E80080FFFCCF80911A0136C080917F
:103BD000CC028132D9F58091D0029091D102892B0B
:103BE000A9F58091E800877F8093E8000E941B2060
:103BF0008091CE0280931A010C946F078091CC02C1
:103C0000813221F58091E800877F8093E8000E944F
:103C10001B208091CF0280939F0208958091CC0257
:103C2000813AA1F48091E800877F8093E800809139
:103C3000E80080FFFCCF80919F028093F10080918B
:103C4000E8008E778093E8000C941B20089584B7D9
:103C5000877F84BF0FB6F894A89580916000886133
:103C600080936000109260000FBE90E080E80FB675
:103C7000F89480936100909361000FBE0C94B21B86
:103C80000E946D200E94CA20E2EEF0E080818460F4
:103C9000808378940C945F238EE091E00C947C1ADE
:103CA0008091CB028530A9F48091CB02853079F4E4
:103CB0000E94031C8091C9028823B1F30E94C41B97
:103CC000882391F30E94C61E0E946F07EDCF0C94CB
:103CD0002E1C089508950C946D1E292F3327233030
:103CE0003105C9F060F42130310581F02230310511
:103CF00009F044C08BE390E024E333E043C0213279
:103D00003105E1F02232310549F138C082E190E01D
:103D10002FE633E037C099278130910549F028F02C
:103D2000029761F5E6E1F3E005C0E0E3F3E002C0ED
:103D3000E2E2F3E0849190E09F0124C061157105F7
:103D400041F061307105D1F489E090E02FE533E076
:103D500019C089E090E026E433E014C061157105D4
:103D600041F06130710551F486EB90E021E833E0D9
:103D700009C080E490E027E334E004C080E090E0F4
:103D800020E030E0FA0131832083089580E189BD8D
:103D900082E189BD09B400FEFDCF8091D8008F7DFE
:103DA0008093D8008091E00082608093E000809151
:103DB000E00081FDFCCF0895CF92DF92EF92FF9259
:103DC0000F931F93CF93DF93EC018B017A010E9435
:103DD0003A20811133C0E114F10439F0F7018081F8
:103DE0009181081B190BC80FD91FC12CD12C0115AB
:103DF000110519F18091E80085FD16C08091E80059
:103E00008E778093E800E114F10449F0F701808196
:103E10009181C80ED91ED182C08285E00FC00E9458
:103E20003A20882321F30AC089918093F100015040
:103E30001109FFEFCF1ADF0ADACF80E0DF91CF91CF
:103E40001F910F91FF90EF90DF90CF9008952091F8
:103E5000D2023091D3022617370748F06115710559
:103E600039F42091E8002E772093E80001C0B901D1
:103E7000FC0120E06115710579F18091CB02882366
:103E8000F1F18530F1F18091E80083FD3CC0809133
:103E9000E80082FD2EC08091E80080FFEBCF2091EA
:103EA000F3008091F20090E0922B6115710551F0C2
:103EB0008830910538F421912093F1006150710907
:103EC0000196F3CF21E0089709F020E08091E80007
:103ED0008E778093E800CECF2111CFCF0AC080919A
:103EE000CB02882361F0853061F08091E80083FD8A
:103EF0000AC08091E80082FFF2CF80E0089582E05E
:103F0000089583E0089581E008952091D2023091D0
:103F1000D3022617370748F06115710539F420914F
:103F2000E8002E772093E80001C0B901FC0120E0F1
:103F30006115710591F18091CB02882309F440C08D
:103F4000853009F43FC08091E80083FD3DC0809139
:103F5000E80082FD2FC08091E80080FFE9CF20912A
:103F6000F3008091F20090E0922B6115710559F0F9
:103F70008830910540F424912093F10031966150EE
:103F800071090196F2CF21E0089709F020E08091B5
:103F9000E8008E778093E800CBCF2111CCCF0AC008
:103FA0008091CB02882361F0853061F08091E80038
:103FB00083FD0AC08091E80082FFF2CF80E008957F
:103FC00082E0089583E0089581E00895982F973066
:103FD00068F59093E900981739F07091EC00209102
:103FE000ED005091F00003C0242F762F50E021FD0A
:103FF00002C09F5FECCF3091EB003E7F3093EB002F
:104000003091ED003D7F3093ED003091EB00316059
:104010003093EB007093EC002093ED005093F00090
:104020002091EE0027FDE5CF80E008958F7080930A
:10403000E90081E008958091CC0287FF11C0809152
:10404000E80082FD05C08091CB028111F8CF11C03C
:104050008091E8008B770BC08091CB02882349F0D8
:104060008091E80080FFF8CF8091E8008E77809300
:10407000E80008952091E4003091E50095E6409134
:10408000EC00842F817040FF23C08091E80080FD08
:104090001DC08091CB02882399F0853099F08091E2
:1040A000EB0085FD11C04091E4005091E50024171C
:1040B000350729F3915011F09A01E1CF84E008957A
:1040C00082E0089583E0089581E0089580E00895F6
:1040D0004091E80042FFDDCF08950E94DB200E945E
:1040E000E320E0EEF0E0808181608083E8EDF0E0A5
:1040F00080818F77808319BCA7EDB0E08C918E7F93
:104100008C9380818F7E80831092CA0208950F93D2
:104110001F93CF93DF930E94DB200E94E320C8ED22
:10412000D0E088818F7788838881806888838881C0
:104130008F7D888319BC1092CB021092C702109217
:10414000C9021092C80200EE10E0F80180818B7F56
:10415000808388818160888342E060E080E00E9403
:10416000E61FE1EEF0E080818E7F8083E2EEF0E0FA
:10417000808181608083808188608083F801808174
:104180008E7F8083888180618883DF91CF911F91AA
:104190000F910895E8EDF0E080818F7E8083E7ED58
:1041A000F0E080818160808384E082BF81E0809341
:1041B000CA020C948720E8EDF0E080818E7F808336
:1041C0001092E20008951092DA001092E100089532
:1041D0001F920F920FB60F9211242F933F934F937C
:1041E0005F936F937F938F939F93AF93BF93EF935F
:1041F000FF938091E10082FF0BC08091E20082FF7B
:1042000007C08091E1008B7F8093E1000E945E23D4
:104210008091DA0080FF1FC08091D80080FF1BC012
:104220008091DA008E7F8093DA008091D90080FF40
:104230000DC080E189BD82E189BD09B400FEFDCFDA
:1042400081E08093CB020E94301D05C019BC109202
:10425000CB020E943E1D8091E10080FF19C0809139
:10426000E20080FF15C08091E2008E7F8093E20023
:104270008091E20080618093E2008091D8008062AA
:104280008093D80019BC85E08093CB020E94431D27
:104290008091E10084FF30C08091E20084FF2CC057
:1042A00080E189BD82E189BD09B400FEFDCF809126
:1042B000D8008F7D8093D8008091E1008F7E80931D
:1042C000E1008091E2008F7E8093E2008091E20025
:1042D00081608093E2008091C702882311F084E01E
:1042E00007C08091E30087FD02C081E001C083E048
:1042F0008093CB020E944B1D8091E10083FF29C077
:104300008091E20083FF25C08091E100877F809348
:10431000E10082E08093CB021092C7028091E1001D
:104320008E7F8093E1008091E2008E7F8093E20097
:104330008091E20080618093E20042E060E080E0F2
:104340000E94E61F8091F00088608093F0000E9438
:10435000411DFF91EF91BF91AF919F918F917F91FF
:104360006F915F914F913F912F910F900FBE0F90E2
:104370001F9018951F920F920FB60F9211242F9332
:104380003F934F935F936F937F938F939F93AF93DD
:10439000BF93CF93DF93EF93FF93C091E900CF706A
:1043A0008091EC00D82FD17080FDD0E81092E90008
:1043B0008091F000877F8093F00078940E94FE2126
:1043C0001092E9008091F00088608093F000CD2B7E
:1043D000CF70C093E900FF91EF91DF91CF91BF9132
:1043E000AF919F918F917F916F915F914F913F918D
:1043F0002F910F900FBE0F901F9018951F93CF9382
:10440000DF93CDB7DEB7AA970FB6F894DEBF0FBE25
:10441000CDBFECECF2E08091F100819322E0E43D2D
:10442000F207C9F70E94691D8091E80083FF2EC141
:104430008091CC029091CD02492F50E04A30510535
:1044400008F024C1FA01E759FF4F0C94D4238038B7
:1044500021F0823809F01AC108C08091C8029091F9
:10446000C902992389F082600FC08091D0028F70B9
:10447000873008F00BC18093E9008091EB0085FB49
:10448000882780F91092E9009091E800977F909337
:10449000E8008093F1001092F100D1C0282F2D7F09
:1044A00009F0F4C0882319F0823061F0EFC08091E8
:1044B000CE02813009F0EAC0933009F080E08093A9
:1044C000C9022EC08091CE0281112AC08091D002F3
:1044D0008F702FEF280F263008F0D8C08093E900A6
:1044E0002091EB0020FF1CC0933021F48091EB0061
:1044F000806214C09091EB0090619093EB0021E0FA
:1045000030E0A90102C0440F551F8A95E2F740939D
:10451000EA001092EA008091EB0088608093EB0043
:104520001092E9008091E800877F8093E8000E9464
:104530001B20ACC08111AAC01091CE021F778091C0
:10454000E3008078812B8093E3008091E800877FEF
:104550008093E8000E941B208091E80080FFFCCF40
:104560008091E30080688093E300111102C082E033
:1045700001C083E08093CB0289C08058823008F06C
:1045800085C08091CE029091CF028C3D53E095077B
:1045900079F583E08A838AE289834FB7F894DE0154
:1045A000139620E03EE051E2E32FF0E050935700F5
:1045B000E49120FF03C0E295EF703F5FEF708E2F14
:1045C00090E0EA3010F0C79601C0C0968D939D939D
:1045D0002F5F243149F74FBF8091E800877F809398
:1045E000E8006AE270E0CE0101960E94271F16C023
:1045F0006091D0027091D102AE014F5F5F4F0E9477
:104600006B1EBC01892B09F441C09091E800977F93
:104610009093E80089819A810E94851F8091E8002B
:104620008B778093E80032C0803881F58091E80074
:10463000877F8093E8008091C7028093F10080918A
:10464000E8008E7772CF811121C08091CE029091C7
:10465000CF0299270297D4F48091E800877F809356
:10466000E8008091CE028093C7020E941B208091B7
:10467000C702811106C08091E30087FD02C081E07E
:1046800001C084E08093CB020E94551D8091E80018
:1046900083FF0AC08091E800877F8093E8008091C3
:1046A000EB0080628093EB00AA960FB6F894DEBF11
:1046B0000FBECDBFDF91CF911F9108950895CF9385
:1046C0008091CB028823A1F0C091E900CF70909136
:1046D000EC00892F817090FD80E8C82B1092E900D2
:1046E0008091E80083FD0E94FE21CF70C093E90015
:1046F000CF910895DB018F939F930E94E923BF918F
:10470000AF91A29F800D911DA39F900DB29F900D20
:1047100011240895AA1BBB1B51E107C0AA1FBB1F90
:10472000A617B70710F0A61BB70B881F991F5A953D
:10473000A9F780959095BC01CD01089597FB072EB0
:1047400016F4009407D077FD09D00E948A2307FC55
:1047500005D03EF4909581959F4F08957095619591
:104760007F4F0895A1E21A2EAA1BBB1BFD010DC0AD
:10477000AA1FBB1FEE1FFF1FA217B307E407F50711
:1047800020F0A21BB30BE40BF50B661F771F881FED
:10479000991F1A9469F760957095809590959B0183
:1047A000AC01BD01CF010895EE0FFF1F0590F491FC
:1047B000E02D0994A29FB001B39FC001A39F700D8B
:1047C000811D1124911DB29F700D811D1124911D19
:1047D00008950E94DA23A59F900DB49F900DA49F89
:1047E000800D911D11240895FB01DC0104C08D9101
:1047F0000190801921F441505040C8F7881B990B53
:104800000895F999FECF92BD81BDF89A992780B598
:104810000895A8E1B0E042E050E00C943524262F42
:10482000F999FECF92BD81BDF89A019700B40216A6
:1048300039F01FBA20BD0FB6F894FA9AF99A0FBE54
:1048400008950396272F0E9410240E940F24252FDD
:104850000E941024242F0C9410240196272F0E94CC
:1048600010240C940F24DC01CB01FC01F999FECF3C
:1048700006C0F2BDE1BDF89A319600B40D924150E8
:0A4880005040B8F70895F894FFCFF8
:10488A00C8002102280850011E0A14010601991CB9
:10489A00BC1C9D1C2C1D281D9C1C01E200E900EA81
:1048AA0000B500B600B700CD008301CC008A0192A2
:1048BA000194012102230224022502260227022A48
:1048CA0002B300B4006F007000818283E200E90045
:1048DA00EA00B500B600B700CD008301CC008A011A
:1048EA0092019401210223022402250226022702B0
:1048FA002A02B300B4006F00700081828393929100
:0E490A0090946697C63436323331F7F6F5F4E2
:00000001FF
